:1070000055C000007FC000007DC000007BC00000B4
:1070100079C0000077C0000075C0000073C0000098
:1070200071C000006FC000000CC200006BC0000007
:1070300069C0000067C0000065C0000063C00000B8
:1070400061C000005FC000005DC000005BC00000C8
:1070500059C0000057C0000055C0000053C00000D8
:1070600051C000004FC000004DC000004BC00000E8
:1070700049C0000047C0000045C0000043C00000F8
:1070800041C000003FC000003DC000003BC0000008
:1070900039C0000037C0000035C0000033C0000018
:1070A00031C000002FC000002DC0000011241FBE01
:1070B000CFEFDAE0DEBFCDBF04B603FE0EC0809195
:1070C00054019091550182349C4D39F41092550130
:1070D00010925401E0E0F0E0099511E0A0E0B1E089
:1070E000E2EEF7E702C005900D92AA34B107D9F796
:1070F00021E0AAE4B1E001C01D92A435B207E1F796
:1071000002D06DC37DCF84B7877F84BF88E10FB67F
:10711000F89480936000109260000FBE81E085BFFC
:1071200082E085BF71D1789480910001882311F0AD
:107130003BD3FACF8091E00081608093E00082E44D
:107140009CED90935501809354012CE088E190E0F0
:107150000FB6F894A895809360000FBE209360004E
:10716000FFCF42E361EC81E0E1C080914C018F7779
:10717000813209F060C080914D01893009F05BC017
:107180008091E800877F8093E8008091E80082FF8B
:10719000FCCF3091F1002091F100832F922F8F3F8F
:1071A0002FEF920719F4109200013FC023E0FC0179
:1071B00020935700E89507B600FCFDCF20E030E0B3
:1071C00061E07091F3004091F20050E0572B452BA5
:1071D000D9F0E091F1007091F1004E2F572FF90195
:1071E000EE0FFF1FE80FF91F0A0160935700E895A3
:1071F00011242F5F3F4F2034310519F725E0FC01A2
:1072000020935700E8950AC04091E8004B774093DF
:10721000E8004091E80042FFFCCFDBCF07B600FC5E
:10722000FDCF81E180935700E8958091E8008B774E
:107230008093E8008FC00895913049F0923061F05A
:10724000913279F489E090E023E131E00EC082E1EF
:1072500090E023E231E009C082E290E021E031E0F9
:1072600004C085E190E025E331E0FA013183208319
:10727000089520915201309153012617370748F0A5
:107280006115710539F42091E8002E772093E8000C
:1072900001C0B901FC0120E061157105A1F18EB3B7
:1072A0008823F1F18530F1F18091E80083FD3CC045
:1072B0008091E80082FF06C08091E80082FF26C02E
:1072C00080E008958091E80080FFE6CF2091F300F0
:1072D0008091F20090E0922B6115710551F0883099
:1072E000910538F421912093F100615071090196C4
:1072F000F3CF21E0089709F020E08091E8008E7735
:107300008093E800C9CF2111CACFD6CF8EB388238E
:1073100039F0853039F08091E80083FFCDCF04C08B
:1073200082E0089583E0089581E008958F7080934E
:10733000E900EBEEF0E0808181608083EDEEF0E02B
:1073400010826093EC0040838091EE00881F8827B4
:10735000881F089580914C0187FD05C08091E80049
:1073600080FF0DC010C08091E80082FD04C08EB384
:107370008111F9CF08958091E8008B7707C08EB313
:107380008111ECCF08958091E8008E778093E8001A
:1073900008950F931F93CF93DF9346D04DD0C8ED40
:1073A000D0E088818F77888388818068888388810E
:1073B0008F7D888319BC1EBA10924A0100EE10E03E
:1073C000F80180818B7F808388818160888342E09F
:1073D00060E080E0ABDFE1EEF0E080818E7F8083D3
:1073E000E2EEF0E08081816080838081886080832C
:1073F000F80180818E7F8083888180618883DF911E
:10740000CF911F910F910895E8EDF0E080818F7E7C
:107410008083E7EDF0E080818160808384E082BF3B
:1074200081E080934B01B5CFE8EDF0E080818E7F65
:1074300080831092E20008951092DA001092E10029
:1074400008951F920F920FB60F9211242F933F931E
:107450004F935F936F937F938F939F93AF93BF935C
:10746000EF93FF938091DA0080FF19C08091D800DC
:1074700080FF15C08091DA008E7F8093DA008091C2
:10748000D90019BC80FF09C082E089BD09B400FEA3
:10749000FDCF81E08EBB87D102C01EBA84D180911E
:1074A000E10080FF17C08091E20080FF13C080914F
:1074B000E2008E7F8093E2008091E2008061809301
:1074C000E2008091D80080628093D80019BC85E0EA
:1074D0008EBB69D18091E10084FF2DC08091E200D4
:1074E00084FF29C019BC82E089BD09B400FEFDCF2C
:1074F0008091D8008F7D8093D8008091E1008F7EAD
:107500008093E1008091E2008F7E8093E200809181
:10751000E20081608093E20080914A01882311F0AB
:1075200084E007C08091E30087FF02C083E001C0D0
:1075300081E08EBB38D18091E10083FF21C0809132
:10754000E20083FF1DC08091E100877F8093E1000E
:1075500082E08EBB10924A018091E1008E7F809381
:10756000E1008091E2008E7F8093E2008091E20052
:1075700080618093E20042E060E080E0D7DE13D1DA
:10758000FF91EF91BF91AF919F918F917F916F91FB
:107590005F914F913F912F910F900FBE0F901F90D1
:1075A00018951F93CF93DF9300D0CDB7DEB7ECE4EF
:1075B000F1E08091F100819381E0E435F807C9F7AB
:1075C000D4DD8091E80083FFDAC090914C01809176
:1075D0004D01853009F465C030F4813059F168F00F
:1075E000833041F1CCC0883009F49CC0893009F463
:1075F000ABC0863009F0C3C075C0903881F09238B6
:1076000009F0BDC0809150018F708093E900909186
:10761000EB0095FB992790F91092E90001C090E0EA
:107620008091E800877F8093E8009093F1001092AA
:10763000F10083C0292F2D7F09F0A1C0923009F0FD
:107640009EC090914E01911126C0209150012F7043
:1076500009F495C02093E9009091EB0090FF1BC0C6
:10766000833021F48091EB00806213C08091EB00A5
:1076700080618093EB0081E090E0022E01C0880FD2
:107680000A94EAF78093EA001092EA008091EB00F6
:1076900088608093EB001092E9008091E800877F7A
:1076A0004FC091116CC010914E011F778091E30083
:1076B0008078812B8093E3008091E800877F80931E
:1076C000E80048DE8091E80080FFFCCF8091E30075
:1076D00080688093E300112311F083E001C082E011
:1076E0008EBB4DC09058923008F049C0AE014F5F3C
:1076F0005F4F6091500180914E0190914F019CDD50
:10770000009709F43CC02091E800277F2093E8000F
:10771000BC0189819A81ADDD8091E8008B778093EF
:10772000E8002DC0903859F58091E800877F80935C
:10773000E80080914A018093F1008091E8008E7703
:107740008093E80007DE1BC0911119C090914E0193
:107750009230A8F48091E800877F8093E8009093AE
:107760004A01F8DD80914A01811104C08091E30053
:1077700087FF02C084E001C081E08EBBF2DC809113
:10778000E80083FF0AC08091E800877F8093E800CB
:107790008091EB0080628093EB000F900F90DF915F
:1077A000CF911F9108950895CF938EB38823A9F0A8
:1077B0008091E9008F709091EC0090FF02C090E8FA
:1077C00001C090E0C92FC82B1092E9008091E80019
:1077D00083FDE7DECF70C093E900CF910895F89460
:0277E000FFCFD9
:1077E20001090222000101008032090400000103A4
:1077F2000000000921110100012215000705810383
:107802004000051201100100000008EB036720018F
:10781200000000000106DCFF09FBA10109021500BE
:0A78220025FF75089682009102C050
:040000030000700089
:00000001FF
